:020000040000FA
:06000000B8EF08F0120049
:06100000B8EF08F0120039
:061008007CEF08F012006D
:061018007EEF08F012005B
:02102A000000C4
:04102C002A0EF66E24
:10103000100EF76E000EF86E00010900F550656F96
:101040000900F550666F03E1656701D03DD00900E6
:10105000F550606F0900F550616F0900F550626F3F
:1010600009000900F550E96E0900F550EA6E090023
:1010700009000900F550636F0900F550646F09001D
:101080000900F6CF67F0F7CF68F0F8CF69F060C0DD
:10109000F6FF61C0F7FF62C0F8FF0001635302E191
:1010A000645307E00900F550EE6E6307F8E2640749
:1010B000F9D767C0F6FF68C0F7FF69C0F8FF000105
:0A10C0006507000E665BBFD7120043
:0610CA000FD88170817255
:1010D0008174817682B002D08A8C01D08A9CC80E3D
:1010E000E66E91EC08F0E552F1D70F0EC16E050ED9
:1010F000816E936A948012000DD81100D8CFE4FF5E
:10110000E0CFE4FFE46E06D8E550E5CFE0FFE5CFA1
:10111000D8FF1000DACFE4FFE652E552E5CFDAFF60
:021120001200BB
:0E112200FF0EE350036EEF0E01D0F30EE76EEA
:10113000E72E98EF08F00C0E026EE76AE72E9EEF9E
:1011400008F0022E9DEF08F0032E96EF08F0120033
:10115000000EF36E00EE00F0080E01D81200EA60F7
:1011600002D0EE6AFCD7F350E9601200EE6AFCD7B9
:1011700013EE00F023EE00F0F86A019C16EC08F084
:0C118000C6EC08F065EC08F0FBD712008C
:02118C0012004F
:00000001FF
